:10000000370101007128A948730000008280148123
:10001000988133E6E60009C685050505E389E6FE15
:1000200013351600828052B82A84452C2A947524F0
:10003000E36F85FE52BE8AB8792425C113044006B9
:1000400093045006130940079309300619A0A52C04
:1000500029C50145712C0808C1450A86C1468D2C69
:1000600003450101E31585FE03451101E31195FEEA
:1000700003452101E31D25FD03453101E31995FCED
:1000800003454101E31535FD03455101E31125FD0C
:10009000034561014DFD05458ABE0545912C8ABC8D
:1000A000FAB81305203319241305803401241304EE
:1000B000A036930500372285112413094037930594
:1000C00090374A85E52A130AD037930520385285A0
:1000D000F522112C930C4006930450069309400717
:1000E000930A3006130D8041930D4042930B7042EA
:1000F00013055038652A0545E52A1305B0387D22D9
:10010000D92221C50145ED220808C1450A86C1460C
:10011000C12203450101E31595FF03451101E311D8
:1001200095FE03452101E31D35FD03453101E3192A
:1001300095FC03454101E31555FD03455101E311CC
:1001400035FD034561014DFD21A0054555224DBFFB
:100150001305C039A12A0145612A4A859305D03B80
:10016000B12A1305003C992222859305A03CB922AF
:100170001305103D252A9522130B3500B92AE36F8C
:1001800065FF22859305103F152A1305003E392A85
:10019000A922130B15009122E36F65FF22859305B9
:1001A000C03E292A1305503F1122052A130B550082
:1001B0002D22E36F65FF52859305704001221305E0
:1001C000C040ED20192A130B4500012AE36F65FF9B
:1001D000192A3D4B09A80545212A0145112A7D1BF5
:1001E0001375FB0F3DC9137CFB0F6A85C120628527
:1001F00055286E856528D520130C1500F928E36F66
:1002000085FFD12069D90145E5200808C1450A8646
:10021000C1467D2803450101E31595FF0345110102
:10022000E31195FE03452101E31D35FD0345310131
:10023000E31995FC03454101E31555FD03455101C3
:10024000E31135FD034561014DFD5D2069285E85A3
:10025000B128614B1375FB0F59F51305C043B92045
:100260004A85930590379928130570448120B5205D
:10027000130B15009D20E36F65FF52859305203811
:100280003528130520451D208928130B2500B12092
:10029000E36F65FF2285930500370D201305C045E8
:1002A0003120B9B585487300000082809148730001
:1002B00000008280AD48730000008280930810081F
:1002C0007300000082809308500873000000828051
:1002D00093087008730000008280732510C082802C
:1002E000732500C08280930860087300000082803C
:1002F0000589F322008093920248B3E2A200739032
:100300000280828095487300000082809308000874
:10031000730000008280A14873000000828093086F
:1003200030087300000082809308400873000000CA
:100330008280554B205261696C726F6164204372F8
:100340006F7373696E670A00666F72205256436F4F
:100350006E74726F6C6C65720A496E697469616C57
:10036000697A696E672048570A006C69676874008B
:100370004F46460062656C6C006F6666006761748C
:10038000650075700049646C650A004C69676874A3
:100390007765696768743A204F6E0A005472616924
:1003A0006E2064657465637465640A4C696768747B
:1003B0007765696768743A204F66660A006F6E0059
:1003C00042656C6C3A204F6E0A0059454C4C4F57B1
:1003D000004C696768743A2059656C6C6F770A0045
:1003E0004C696768743A205265640A00464C415370
:1003F00048524544004C696768743A20466C617302
:1004000068205265640A00646F776E004761746506
:100410003A20446F776E0A0054696D656F757420D9
:10042000696E2000730A0054696D652072657365FA
:100430007420627920747261696E0A0054696D6576
:1004400064206F75740A0042656C6C3A204F6666D2
:100450000A00476174653A2055700A004C69676864
:08046000743A204F66660A00A1
:00000001FF
